:020000040800F2
:1000000000020020010100080501000807010008A6
:10001000090100080B0100080D01000800000000A4
:100020000000000000000000000000000F010008B8
:10003000110100080000000013010008150100086C
:100040001701000817010008170100081701000830
:100050001701000817010008170100081701000820
:100060001701000817010008170100081701000810
:100070001701000817010008170100081701000800
:1000800017010008170100081701000817010008F0
:1000900017010008170100081701000817010008E0
:1000A00017010008170100081701000817010008D0
:1000B00017010008170100081701000817010008C0
:1000C00017010008170100081701000817010008B0
:1000D00017010008170100081701000817010008A0
:1000E000170100081701000817010008DFF80CD0FD
:1000F00000F0B4F800480047950100080002002015
:1001000005480047FEE7FEE7FEE7FEE7FEE7FEE7FD
:10011000FEE7FEE7FEE7FEE7ED00000800BF122065
:100120001249086000BF00BF1148806940F0040018
:100130000F4988614FF011300E4908600E480F4991
:10014000C1F804080A48806940F00800084988613D
:100150000B480C4908600C480849C1F8040C00BF62
:1001600070470A4870470A48704700000020024064
:100170000010024000080140011001000000014091
:1001800000001011000C0140008081100051250278
:1001900000A24A04FFF7C2FF2C48006840F4205038
:1001A0002B49C1F80C0C4FE02A48006810F4006F8E
:1001B00010D12948006840F60F1140EA0100244997
:1001C000C1F80C080846D0F80C0C40F06000C1F8EB
:1001D0000C0C0FE02048006840F60F1120EA0100E7
:1001E0001B49C1F80C080846D0F80C0C20F0600040
:1001F000C1F80C0C1748006810F4005F12D11648C3
:10020000006841F2F00140EA01001149C1F80C0810
:100210000E48006849F2800140EA01000C49C1F82B
:100220000C0C11E00C48006841F2F00120EA0100DA
:100230000749C1F80C080548006849F2800120EA26
:1002400001000349C1F80C0CAEE700000C0C0140A2
:1002500000000140080C01400C080140064C074D0D
:1002600006E0E06840F0010394E807009847103486
:10027000AC42F6D3FFF73EFFA0020008B002000830
:1002800002E008C8121F08C1002AFAD1704770475F
:10029000002001E001C1121F002AFBD170470000BD
:1002A000B0020008000000200002000090020008D8
:04000005080000ED02
:00000001FF
